:020000040000FA
:100000001C0AE2012008100822081208320813080E
:100010008702060F4307060F2700000826000A0C78
:10002000130A26001E0C2900B20C2100010243070E
:10003000160AE902140A0008060C0200080C060061
:1000400066006700B20C210008096607220A010257
:100050004307240A300C0E09210C0E09220C0E094C
:10006000210C0E09300C0E09210C0E09220C0E0970
:10007000210C0E090702010928004000110908029D
:100080001109400011090802110940001109080274
:100090001109DC0C2A00050C2B0066075D0A010C17
:1000A00013090A024306EB00EA000A020B014307A8
:1000B0004D0A6600060203000000010C13096606E3
:0400C0004D0A220AB9
:0400C4000008000828
:021FFE00EA0FE8
:00000001FF
